:107000006BC00000AAC000008EC000008CC0000051
:107010008AC0000088C0000086C0000084C0000054
:1070200082C0000080C000007EC000007CC0000064
:107030007AC0000078C0000076C0000074C0000074
:1070400072C0000070C000006EC000006CC0000084
:107050006AC0000068C0000066C0000064C0000094
:1070600062C0000060C00000EC2DFD2DB7B6B0FC82
:10707000FDCF27BFE895B7B6B0FCFDCF21E1B7B68D
:10708000B6FCF4CF08950902120001010080320914
:10709000040000000000000012011001FF000008C1
:1070A000C016DC050201010200010E035500530069
:1070B00042006100730070001C03770077007700C6
:1070C0002E00660069007300630068006C002E00EB
:1070D000640065000403090411241FBECFEFD8E04B
:1070E000DEBFCDBF24B7D8E0CEEF39913833399128
:1070F00009F03FEF30933C0120933B0111E0A0E009
:10710000B1E0E4E8F8E702C005900D92A630B107BF
:10711000D9F721E0A6E0B1E001C01D92AB33B20780
:10712000E1F785D1ADC36CCFA82FB92F80E090E0F7
:1071300041E050EA609530E009C02D918227979593
:10714000879510F084279527305EC8F36F5FA8F30A
:107150000895EADF8D939D930895CF93CFB7CF9392
:10716000DF93C3954B9BE9F74B9B0BC04B9B09C02F
:107170004B9B07C04B9B05C04B9B03C04B9B01C067
:1071800089C06F93C0911E01DD27CB5DDE4F2F9329
:1071900065E54B9B03C02F916F91E6CF0F931F9333
:1071A0004F9320E040E15F9309B10C7003FB27F996
:1071B0003F9350E03BE039C01C7040642F77012FB3
:1071C0005F5F1EC0406819B11C702F7752501FC0FE
:1071D000406409B12F770C70D1F15F5F00C023C00C
:1071E000406219B12F771C7091F15F5F00C025C01C
:1071F0000C701027515012F45D5F0000115027955C
:107200002C3F19B1C8F61C700127015027952C3F5F
:10721000C8F64227499309B10C7010274F731150DB
:1072200027952C3FA8F64695469519B11C7079F024
:107230000127015027952C3F98F66B5A60F3315087
:1072400009B1B0F600C011E01CBB002717C03B50CD
:107250003195C31BD04011E01CBB0881033CF9F001
:107260000B34E9F020911C011981110F1213EDCF9D
:10727000093651F10D3211F0013E39F70093230127
:107280003F915F914F911F910F912F916F91CCB3CF
:10729000C0FD67CFDF91CF91CFBFCF9118952091DF
:1072A0002301222369F310912101112339F5343090
:1072B0003AF13093210120931D0110911E013BE012
:1072C000311B30931E011CC0009121010130B4F428
:1072D0000AE53091010134FD14C000930101C1E1C0
:1072E000D1E013C0052710E000C000000BB91AC0A0
:1072F000052710E0221F1DC010E021C04AE502C092
:1073000032ED432FC4E1D0E032E01AB11C605B9A49
:107310000BB11AB95CE020E865E320FF05270BB943
:10732000279517951C3FF0F66695B8F7B1F720FF43
:1073300005270BB9279517951C3FD0F6279517956C
:1073400017FF052700001C3F0BB9B0F629913A95AD
:1073500019F7037F10912201110FC651D0400BB9CC
:1073600011F010931C0111E01CBB08601AB1137FCF
:10737000402F437F54E05A95F1F70BB91AB94BB936
:107380007FCFDC0113964C91139714963C91149780
:1073900013968D919C911497982789279827129678
:1073A0002C911297203339F43370E32FF0E0EE5F25
:1073B000FE4F80810895283561F489E0E1E0F0E036
:1073C000442371F089E0E3E0F0E0483049F080E0E8
:1073D0000895203579F4411107C089E0F0E0E0E03C
:1073E000809357008491089589E0E2E0F0E048300E
:1073F00071F7F6CF203229F4880F991FFC01849190
:107400000895283229F4FC01EE0FFF1F3196F7CFC3
:10741000203A09F41FC2203C21F415966C9122D227
:10742000D6CF2F3FA1F681EF80930F01D0CF1AB8AE
:1074300080E28BB981E085BF82E085BFE0E0F1E7C3
:10744000A89531978040E1F780913B01877F21F437
:1074500080913C01882371F04D9B0CC0F894539AA5
:107460001BB81DBA1092690081E085BF15BEF0E01F
:10747000E0E009958EEF80930F0114BE0FB6F894EB
:10748000A8958091600088618093600010926000F0
:107490000FBE80916900826080936900E89A539AD8
:1074A0008CE0E0E0F5E3A89531978040E1F7539850
:1074B000789410912101135017FD5AC080911E013C
:1074C000CCE0D0E0C81BD109CB5DDE4F80911D011F
:1074D0008D3209F00BC1183009F048C083EC80935D
:1074E00011018AE580930101109210013881832FE8
:1074F00080769981882309F49BC046E051E050933F
:10750000200140931F01933069F4CE013ADF80934C
:10751000090184E09F81911127C09E81981720F571
:10752000892F22C0953009F4DFC09A3009F4DCC0FD
:107530008CEF890F863008F070C04A815B815093D0
:107540000E0140930D01993009F46EC08E81809335
:107550000C012D81227020930B0190930A0137FFBB
:107560008FEF90E890931001809300011092210119
:107570008091010184FF36C0C0910001CF3F91F19D
:107580008C2FC93008F088E09C2F981B9093000145
:107590009091110128E8922790931101CC23B1F02A
:1075A0004091100147FF2FC190910C01C82F9817EF
:1075B00008F4C92F9C1B90930C01D0900A01D0E0D5
:1075C00082E1E82E81E0F82EDC1304C16C2F82E109
:1075D00091E0BFDDCC5FCC3019F08FEF80930001DC
:1075E000C093010184E199B19C7031F48150D9F7C5
:1075F0001092220110921C0180910F01803108F439
:107600001EC14D9B05C080910F01805180930F01D9
:1076100080910F0181114DCF21CF80910F019230C8
:1076200029F48E7F80930F0180E074CF8160FACFC0
:107630002A8110921A0191110AC010921B012AE1AD
:1076400031E082E03093200120931F0163CF953019
:1076500029F4209322012AE131E0F4CF963099F504
:107660009B81913059F488E990E7909320018093B1
:107670001F0182E190E4909310014CCF923019F4F5
:1076800086E890E7F2CF9330A9F7211108C084ED86
:1076900090E79093200180931F0184E0EBCF21308D
:1076A00041F488EB90E79093200180931F018CE1D7
:1076B000E1CF2230F9F68AEA90E790932001809397
:1076C0001F018EE0D7CF983059F0993019F42093EC
:1076D0002401C1CF81E09A3009F4BDCF80E0BBCF57
:1076E00024E231E081E0AECF81E014CF809110013F
:1076F00087FF3CCF00910C01011708F4102F011BEC
:1077000000930C01F12CF11628F001112FCF1092EB
:1077100000012CCF80910D0190910E0120910A0162
:10772000273058F069919C012F5F3F4F30930E0135
:1077300020930D0197D0F394E6CF8115904738F749
:10774000F394F394F894E0910D01F0910E012991D6
:10775000399181E0090180935700E89511247894CC
:1077600080910D0190910E01029690930E018093ED
:107770000D018F779927892B51F00111C4CFF11694
:1077800008F4C1CF80910B01882309F4BCCFF89491
:10779000E0910D01F0910E01329783E08093570044
:1077A000E895789407B600FCFDCFF894E0910D01C0
:1077B000F0910E01329785E080935700E895789418
:1077C00007B600FCFDCFF89481E180935700E8955F
:1077D000789499CF00910D0110910E0126E02D159E
:1077E00078F4C80137D0F7018083FFEFEF1AFF0A62
:1077F0000F5F1F4F10930E0100930D01DF5FE4CE6A
:10780000F8018491F0CF90911F0130912001282F31
:10781000290FE92FF32FA2E1B1E046FF0BC09491AD
:107820009D9331962E13FBCFF0932001E0931F011F
:10783000C82FCCCE91919D932E13FCCFF5CF4D99AF
:10784000E7CE80910F01823008F4E2CE80910F01E3
:107850008250DCCEF999FECF92BD81BDF89A99276E
:1078600080B50895262FF999FECF1FBA92BD81BD2C
:1078700020BD0FB6F894FA9AF99A0FBE01960895B2
:04788000F894FFCFAA
:06788400FF5A1E950F00E3
:040000030000700089
:00000001FF
